:1074000080E189BD82E189BD09B400FEFDCF089508
:10741000D3D569F08091E9008F931092E900A8D448
:1074200083FF01C027D58F9187708093E90008956D
:107430008EEF0090E10008220092E1000895F20131
:10744000F999FECFF2BDE1BD0895F9DFF89A80B554
:1074500008C0F5DF1FBA80BD0FB6F894FA9AF99A02
:107460000FBE31962F010895E0E0F0E085919491F0
:107470000196089580EE8BB98BEA34D01092890082
:107480008AEF8093880082E080936F0083E080938E
:107490008100E7E5F7E785913AD0E336E1F781E04F
:1074A0008093D7008AE482BF1092D8001092E20045
:1074B0001092DA001092E10080E808D019BC1EBAE0
:1074C0001092E0006BD489E05CD481E98093D8000D
:1074D0000895A3E6B1E090E81AD08D939A95E1F76C
:1074E000089586E008D010C083E005D08F2F0FD01C
:1074F0008E2F0DD080E05F9A5A9809C005D085E0A4
:10750000FADF05D080FDFDCF5A9A5F9808958EBDB1
:107510008DB587FFFDCF8EB508958FE08221E9F705
:10752000F3DFE3E6F6E090EB5C98892FF0DF80E193
:10753000EEDF5C9A8191EBDF83E68E278F77D1F7C0
:107540009395983B89F70895E3E6F1E094FC38C001
:1075500096FC4FC090FE08958684882011F49924EB
:1075600059C0F894C089D78520E030E080E090E4ED
:10757000AFEFBFEF119688199040E0F72D01BD4F96
:107580008D0127FD13C0E0E0F8E011928EE78193B2
:1075900092E4E11791939AE508F092E4E334C9F795
:1075A00081931082BDDFFE0121969EDF92DFF901FB
:1075B00006D520583F4F040D151D8A9411F715C2AA
:1075C0008301282D60906C0170906B0141D019F4FB
:1075D0008823C1F70895380188243AD0B9F58091FD
:1075E0006A01821709F4830160906E0170906D0149
:1075F000F4CF60906E0170906D012AD059F4882309
:10760000C1F708959FEF95FC03C092FE089591E0A5
:1076100097FB890E662477248301222719D0B1F4C1
:107620008823A1F380916A0136F0881650F48217FE
:1076300030F0213003C0881520F4281710F483019E
:10764000282F60906E0170906D01E8CF3801822E76
:10765000F3014ADF3EDFC3E6D1E0E0E5F7E709905A
:107660008591081621F4E735D1F7088080104CCFBA
:10767000C9E031DFCA95E9F7D0E195FC1EC094FC62
:1076800053C096FC35C0C3E6D2E0E3E6F6E098E0EE
:1076900088E78E0F00840192E817E1F7884F099080
:1076A0000192E817E1F7C858DF4F9A9589F735DF5F
:1076B000C85FD340C33E49F749C0C3E6D6E0EBE517
:1076C000FAE098E08E2F885702900086E817E1F7DD
:1076D00038960A900292E817E1F73897C857D040D9
:1076E0009A9581F71ADFC850DC4FC33E41F72EC090
:1076F000A3EEB6E0E3E6F6E09AE0C6E00D90808106
:107700008025807F802582958193A336B90709F46F
:10771000B2E0E336F90709F4F2E0E336FC0771F76B
:10772000FCDEDA9529F712C0A3EEB9E0E3E6FAE051
:1077300092E00E90829180258F70802582958083C3
:10774000E336F907B1F7E9DEDA9571F7882708958E
:1077500041524455424F59D5F08D14A1C881CFD91B
:10776000F1AF000000FFFFCFCFFFFFFFFFCFCFFF44
:10777000FF0000FE067E7E06FE46565616FE0656A4
:10778000461EFE3F61E9E3FFE3EBE3FFE3EBE3FFCC
:04779000E16B3F006A
:10779400120110010200000841233600010000001C
:1077A400000109023E0002010080320904000001C8
:1077B4000202010005240010010424020405240629
:1077C4000001070582030800FF09040100020A0002
:1077D40000000705040210000107058302100001E0
:1078000011241FBE04B714BE88E18093600010925B
:1078100060008EEF9AE09EBF8DBF222433242101A9
:107820003101410180E88AC00F928F939F931F928C
:107830000FB60F9211244F936F938091DA0080FF5F
:1078400037C023C00F920FB68F939F93EF93FF9390
:1078500088278093850080938400E0E5F1E09281A1
:10786000907261F490818917980B908309F45D9A66
:1078700091818917980B918309F4289A239411F424
:107880008315381EFF91EF9154C08091D80080FF7E
:107890000FC08091DA008E7F8093DA008091D9004A
:1078A00080FF04C0ADDD81E08EBB02C019BC1EBAF2
:1078B0008091E10080FF0BC05ED280FF08C05ED2E5
:1078C0008091D800806202DE19BC85E08EBB809179
:1078D000E10084FF1AC04FD284FF17C091DD809170
:1078E000D8008F7DF3DD8FEEA4DD45D28F7E8160E1
:1078F00048D280915301882331F48091E30087FDC1
:1079000002C081E001C084E08EBB8091E10083FF72
:107910000CC031D283FF09C087EF8BDD82E08EBBC4
:107920001092530185DD2AD239D26F914F910F9079
:107930001F909F918F910FBE0F90189580936100BB
:1079400010926100B1E0B5BF82E085BF87E084B9E5
:1079500081E785B917B8469A10BA80EC81BB84EAF2
:107960008BB984EF8AB980E58CBDBDBDA0E0E4E9A8
:10797000F7E705900D92A035E1F71D92BB30E9F7CE
:1079800001FD09C000FF07C01E9B05C05EDD882306
:1079900012F06ADD51F56EDD78945ADE71F0ABE9D4
:1079A000B7E0E3E6F7E790E105900D929A95E1F7ED
:1079B000A059BF4FE339B9F7B4DD54D029DD809128
:1079C0005201807871F483B180958077369B846012
:1079D0007F997E9B8160982E15DE8110B5DD90FC2D
:1079E00002C0332052F740DD41F3F89489EB7ADD91
:1079F00081E08093E00010926F001092810010925D
:107A000085001092840081E085BF15BE289A289ACF
:107A1000289A5D9A289A0C940000A8D107C05BD1DF
:107A200002C0CAD239F0A4D182FFFBCF85FFF7CFC5
:107A30008091F1000895082E83E099D185FD07C05B
:107A40008ED102C0B9D269F093D180FFFBCF0092F2
:107A5000F10080915201807221F45D9884E6809358
:107A60005001089583D182FF38C180915201807204
:107A700021F4289884E680935101CFDF182F8534B4
:107A800031F422248EE7382EDADC8DE00FC1843504
:107A900011F4C3DFFACF8C34C1F38035B1F38437EE
:107AA00021F484E4C8DF80E001C1813611F489E566
:107AB000FDC0813429F4B1DF582EAFDF482EE5CF69
:107AC000803711F483E5F2C0833539F4E0E5F7E758
:107AD0008591B1DFE735E1F7EAC0863521F481E32E
:107AE000AADF87E3E3C0863781F481E37F9B8E5F63
:107AF0007E9B8F5FA0DF81E41C9B885F369B8C5F41
:107B00001D9B8E5F1E9B8F5FD1C08837A9F485DFD8
:107B100080935201289A84FD28985D9A83FD5D9890
:107B2000289A81FD2898289A82FD2898289A80FD15
:107B3000289887FD8824A9CF8A3649F48FE9DBDCB1
:107B4000C3E0E5DC78DFCA95E1F7DEDCB0C083375F
:107B500031F487E870DF85E96EDF8EE1A7C08536F6
:107B600039F4E0E8F3E73ED2E058F040E0F78DCF9B
:107B7000823631F489E55FDF80E05DDF80E896C022
:107B8000823419F0873609F07DC0332446DFD82FC0
:107B900044DFC82F42DF082F8354843008F085C0AB
:107BA000063411F4440C551CF20110926F00173684
:107BB000B9F4033489F483E098DCA9DC8EB51EBCEB
:107BC0003ADF0DB42197D1F79FDC08C0063411F4D9
:107BD000859101C03ADC2FDF2197C2F72F014AC0FF
:107BE0000334A9F4E11104C07CDC88ED7EDC86DC82
:107BF00078DC82E07ADC11DF0DB48EBDCA95D9F74E
:107C0000319686DC7BDCDA9569F72F0131C00634CA
:107C1000F1F49F01F437D8F4E5D119C0FEDE063443
:107C200061F4C0FB46F0F43728F4182E81E087BFDA
:107C3000E89511243296082E0AC0043439F4DF0185
:107C4000B370AD59B94F8D93319601C002DC2197C5
:107C50002AF7043431F42F01F370FE2B49F461DC70
:107C600007C0063429F42F01F901F43708F4B8D11C
:107C70008DE0E1DE063411F45694479482E080935F
:107C80006F0015C08237E1E049F08634E0E031F062
:107C90008E34E3E019F0813531F4E2E0F0E089E080
:107CA00087BF849103C08B3111F08FE3C4DE83E082
:107CB000BCDB55D095FF03C009C07ED171F058D010
:107CC00080FFFBCF4CD002C077D139F051D080FF7C
:107CD000FBCF84E0AADB8BE743C00895E4E5F1E045
:107CE00067E090915B0180915C01913231F0913AB3
:107CF000E1F58132D1F55ED181C0823271F481919A
:107D0000805B8191844089F580915D0180FD2DC06B
:107D1000F89481E08093E00073CD803231F54AD150
:107D20004BD1E9F08530D9F023D083FD18C082FF14
:107D3000F7CF04C07DDE8193615031F09091F30064
:107D40008091F200892BB1F7C6DF611549F704C0B5
:107D500033D129F0853019F00BD080FFF9CF8EE7B1
:107D60009091E80089238093E800089584E05DDB2A
:107D70008091E80008958091E2000895FCDF8E7FF5
:107D800080618093E200089582E061EC09D083E095
:107D900061E802D084E060E842E103C080E060E096
:107DA00042E043DB81E007D01092ED006093EC00ED
:107DB0004093ED0008959091EB00892B8093EB00A8
:107DC000089560E0923029F0913029F4E0E062E11A
:107DD00002C0E2E16EE3F1E0089580915B01882347
:107DE0004CF402C0E9D0C1F3C3DF82FFFBCF73CFF5
:107DF000E3D091F3BDDF80FFFBCFB1CF40916101B4
:107E0000509162014617510520F0462F611509F483
:107E1000A6DF50E022C0D0D061F1853051F1A8DF5B
:107E200083FD59CFA5DF82FD21C080FF16C03091B0
:107E3000F3002091F20006C081918093F10041503F
:107E40002F5F3F4F411519F028303105A8F350E05E
:107E50002830310509F451E082DF4115E1F6552360
:107E6000D1F604C0A9D029F0853019F081DF82FF56
:107E7000F9CF31CFEBE5F1E0DBDD8193E336E1F7DC
:107E80002DDF76DF83FF91C080915B0190915C01D3
:107E9000913009F170F09330F1F0953009F444C05D
:107EA000963009F456C0983009F460C0993059F7FB
:107EB00067C0823841F780915F01B6DA2091EB000C
:107EC0001092E90077D02295269521702093F10039
:107ED0001092F10052C0882311F08230A1F68F7108
:107EE000823089F680915D018823D1F420915F0171
:107EF000277049F22093E9008091EB0080FF10C0C9
:107F0000933011F480E20BC080E155DF81E0880FEF
:107F10002A95E9F78093EA001092EA0088E04BDFA7
:107F20001092E90047D02AC0882391F410915D0196
:107F300010680FB7F8943ED050DF1ADF80FFFDCFF6
:107F40001093E300103883E009F482E08EBB0FBF8A
:107F50002CC08058823048F580915D0190915E017F
:107F600030DF603011F126D049DF1FC08038E9F4DE
:107F700021D0809153018093F100F1DE2EDF15C0F6
:107F8000882399F490915D01923078F49093530195
:107F900011D023DF80915301882321F48091E300E5
:107FA00091E087FD94E09EBBEFDEE2DE83FF089563
:107FB00080E201DF87EFD4CE8EB388230895A3E655
:107FC000B1E0F437B8F40ED090E40D901D9081E04C
:107FD00087BFE89532969A95C1F71124E058F04092
:107FE00085E001C083E001D081E187BFE89507B655
:067FF00000FCFDCF089526
:067FFA003137E2CFFBDC91
:040000030000740085
:00000001FF
